:0300000002000EED
:20000B00020196758131D2AFD2A912019F80FE12001B80FBC82581C822C92581C97A002215
:20002B00D083D082CF2581F581CFC082C08322CF2581F581CF22FBE493CB22FCE493FB7492
:20004B000193CC22FAE493F9740193CA2229F9E5F03AFA227C00CB30E7011CCB2275F0009B
:20006B0030E70215F022FDE493FF7401934F7004A3A3800C740293B50510740393B5F00A99
:20008B00E493C0E0740193C0E022A3A3A3A380D7FEEBA4FD8EF0ECA4FCEB8EF0A4C5F02C0F
:2000AB002DC5F02211B58EF0ED22C002C001AAF0F97E007D007F11C3E933F9EA33FADF0867
:2000CB00F5F0E9D001D00222ED33FDEE33FEC3ED9BF5F0EE9C40E0ADF0FED380DBBB0001E7
:2000EB0022C333C5F033C5F0DBF722BB000122C3C5F013C5F013DBF722240280022401C595
:20010B00F03400C5F022C394028003C39401C5F09400C5F0223116F4C5F0F4C5F02245F095
:20012B007022042231784024801A3178401E7014801A3178400E7014800A3178500E8004A0
:20014B00318C6008E4F5F022318C60F8E4F5F00422318C40F780ED318C40F170E780ED313C
:20016B008C40E170E780DD318C50E180D7C39BC5F09C20E70720D207C345F02220D2F9D340
:20018B0022C5F0C39C7003E5F09B22758CDC758A000508327421F589748075F025C0E0C00D
:2001AB00F0120D89158115817400F508740075F000F50B85F00C740075F000F50985F00A4F
:2001CB007400F5137400F5147400F5177400F516C2B5C2B47400F590740575F000C0E0C0F8
:2001EB00F01206E115811581120391120C68748875F013C0E0C0F01206E115811581E517CE
:20020B004404F517120432740075F000791E7A00120058741075F027F709A7F0E5174402FA
:20022B00F517120A747459F588740175F00045F0700302026BE5081200687B0A12005F126D
:20024B00012F45F060030202407400F508D2B012026C1207CA120A74120432C2B0020234AF
:20026B0022E51304F51314E51375F0007B017C0012017245F070030202E57400F513E51459
:20028B0004F51414E51604F51614E5174401F517E51675F0007B0A7C0012017245F0700339
:2002AB000202B8740AF516E5174402F517E51475F0007B0A7C0012017245F070030202E52B
:2002CB007400F514E509850AF0120108F50985F00A120116E5174404F51722058105817476
:2002EB000075F00078FD12001FF608A6F078FD12001FE60886F078F912001F86030886048D
:20030B0012012F45F07003020330801678FD12001FE60886F012010818F608A6F012011623
:20032B0080CB020317158115812278FB12001FE6F515E515C2B4C2B5F590D2B500C2B5C43B
:20034B00F590D2B500C2B5740175F000C0E0C0F01202E6158115812278FB12001FE6F51509
:20036B00E515D2B4C2B5F590D2B500C2B5C4F590D2B500C2B5740175F000C0E0C0F0120273
:20038B00E615811581227430F59012042C740A75F000C0E0C0F01206E11581158112042C19
:2003AB00740175F000C0E0C0F01206E11581158112042C740175F000C0E0C0F01206E11569
:2003CB008115817420F59012042C12042C12042C742875F000C0E0C0F01203351581158155
:2003EB00740C75F000C0E0C0F012033515811581740675F000C0E0C0F012033515811581A2
:20040B00740175F000C0E0C0F012033515811581740575F000C0E0C0F01206E115811581DE
:20042B0022D2B500C2B522058105810581E517540475F0007B047C0012014B45F070030221
:20044B000691E51754FBF517740078FE12001FF6748075F000C0E0C0F01203351581158173
:20046B00E509850AF07B107C271200B57B007C0012015345F070030204AFE509850AF07B6D
:20048B00107C271200B52430C5F03400C5F0C0E0C0F012036315811581740178FE12001FD5
:2004AB00F60204BF742075F000C0E0C0F012036315811581E509850AF07B107C271200AF2D
:2004CB0078FC12001FF608A6F008E61200687B0012005F12014B45F060141818E60886F0E9
:2004EB007BE87C031200B57B007C0012014B45F07003020513742075F000C0E0C0F01203D3
:20050B00631581158102053E78FC12001FE60886F07BE87C031200B52430C5F03400C5F058
:20052B00C0E0C0F012036315811581740178FE12001FF678FC12001FE60886F07BE87C03BF
:20054B001200AF18F608A6F008E61200687B0012005F12014B45F060141818E60886F07BB9
:20056B00647C001200B57B007C0012014B45F07003020592742075F000C0E0C0F012036372
:20058B00158115810205BD78FC12001FE60886F07B647C001200B52430C5F03400C5F0C083
:2005AB00E0C0F012036315811581740178FE12001FF678FC12001FE60886F07B647C001274
:2005CB0000AF18F608A6F008E61200687B0012005F12014B45F060141818E60886F07B0A41
:2005EB007C001200B57B007C0012014B45F07003020611742075F000C0E0C0F012036315C1
:20060B0081158102063478FC12001FE60886F07B0A7C001200B52430C5F03400C5F0C0E019
:20062B00C0F01203631581158178FC12001FE60886F07B0A7C001200AF18F608A6F018E6E6
:20064B000886F02430C5F03400C5F0C0E0C0F012036315811581742075F000C0E0C0F012D0
:20066B00036315811581747375F000C0E0C0F012036315811581742075F000C0E0C0F01242
:20068B000363158115811581158115812205810581740075F00078FD12001FF608A6F07842
:2006AB00FD12001FE60886F07B087C0012012F45F070030206DC801678FD12001FE6088620
:2006CB00F012010818F608A6F012011680D10206C3158115812205810581740075F0007868
:2006EB00FD12001FF608A6F078FD12001FE60886F078F912001F860308860412012F45F0EF
:20070B00700302072E801678FD12001FE60886F012010818F608A6F012011680CB12069899
:20072B00020712158115812274FFF590D2B730B7FD20B7FD740175F000C0E0C0F01206E1E9
:20074B0015811581E590540F75F000F51885F019740275F000C0E0C0F01206E1158115813A
:20076B0074FFF590E590540F75F000F51C85F01D740275F000C0E0C0F01206E11581158146
:20078B0074FFF590E590540F75F000F51A85F01BE5188519F07B647C0012009BC0E0C0F097
:2007AB00E51A851BF07B0A7C0012009BD004D0032BC5F03CC5F0251CC5F0351DC5F022E575
:2007CB0017540175F0007B017C0012014B45F07003020968E51754FEF517741275F000790E
:2007EB001E7A00120058741075F000C001C002791E7A00120058E70987F0D007D000F608F9
:20080B00A6F0741075F000791E7A00120058740E75F000C001C002791E7A00120058E709FE
:20082B0087F0D007D000F608A6F0740E75F000791E7A00120058740C75F000C001C00279B8
:20084B001E7A00120058E70987F0D007D000F608A6F0740C75F000791E7A00120058740A0B
:20086B0075F000C001C002791E7A00120058E70987F0D007D000F608A6F0740A75F000790C
:20088B001E7A00120058740875F000C001C002791E7A00120058E70987F0D007D000F60860
:2008AB00A6F0740875F000791E7A00120058740675F000C001C002791E7A00120058E7096E
:2008CB0087F0D007D000F608A6F0740675F000791E7A00120058740475F000C001C0027928
:2008EB001E7A00120058E70987F0D007D000F608A6F0740475F000791E7A0012005874027B
:20090B0075F000C001C002791E7A00120058E70987F0D007D000F608A6F0740275F0007973
:20092B001E7A00120058740075F000C001C002791E7A00120058E70987F0D007D000F608C7
:20094B00A6F0740075F000791E7A00120058C001C002120733D007D000F608A6F022740002
:20096B0075F000791E7A00120058740275F000C001C002791E7A00120058D007D000E6081E
:20098B0086F027C5F00937C5F0C0E0C0F0740475F000791E7A00120058D0F0D0E027C5F011
:2009AB000937C5F0C0E0C0F0740675F000791E7A00120058D0F0D0E027C5F00937C5F0C08C
:2009CB00E0C0F0740875F000791E7A00120058D0F0D0E027C5F00937C5F0C0E0C0F0740A11
:2009EB0075F000791E7A00120058D0F0D0E027C5F00937C5F0C0E0C0F0740C75F000791EFF
:200A0B007A00120058D0F0D0E027C5F00937C5F0C0E0C0F0740E75F000791E7A00120058F4
:200A2B00D0F0D0E027C5F00937C5F0C0E0C0F0741075F000791E7A00120058D0F0D0E0271F
:200A4B00C5F00937C5F0C0E0C0F0741275F000791E7A00120058D0F0D0E027C5F00937C5DA
:200A6B00F07B0A7C001200B5220581058105810581E517540275F0007B027C0012014B4526
:200A8B00F07003020C5FE51754FDF51774C075F000C0E0C0F012033515811581742075F0CA
:200AAB0000C0E0C0F01203631581158112096978FB12001FF608A6F018E60886F0F50D8578
:200ACB00F00E18E60886F0AB0FAC1012015C45F07003020AEA18E60886F0F50F85F0107891
:200AEB00FB12001FE60886F0AB11AC1212016A45F07003020B0B18E60886F0F51185F0129B
:200B0B0078FB12001FE60886F07BE77C0312012F45F0600C18E60886F07B007C0012013D3B
:200B2B0045F07003020BEF78FB12001FE60886F07B647C001200B508F608A6F018E60886B4
:200B4B00F07B007C0012015345F07003020B7518E60886F02430C5F03400C5F0C0E0C0F055
:200B6B0012036315811581020B85742075F000C0E0C0F01203631581158178FB12001FE6BD
:200B8B000886F07B647C001200AF18F608A6F018E60886F07B0A7C001200B52430C5F03483
:200BAB0000C5F0C0E0C0F012036315811581742E75F000C0E0C0F01203631581158178FB13
:200BCB0012001FE60886F07B0A7C001200AF2430C5F03400C5F0C0E0C0F01203631581154E
:200BEB0081020C2F742D75F000C0E0C0F012036315811581742D75F000C0E0C0F012036364
:200C0B0015811581742D75F000C0E0C0F012036315811581742D75F000C0E0C0F0120363D5
:200C2B001581158174DF75F000C0E0C0F012036315811581744375F000C0E0C0F0120363ED
:200C4B0015811581742075F000C0E0C0F0120363158115811581158115811581227480758D
:200C6B00F000C0E0C0F012033515811581744475F000C0E0C0F01203631581158174697550
:200C8B00F000C0E0C0F012036315811581746775F000C0E0C0F012036315811581746975DF
:200CAB00F000C0E0C0F012036315811581745475F000C0E0C0F012036315811581746875D3
:200CCB00F000C0E0C0F012036315811581746575F000C0E0C0F01203631581158174727598
:200CEB00F000C0E0C0F01203631581158174C075F000C0E0C0F012033515811581746D7550
:200D0B00F000C0E0C0F012036315811581743075F000C0E0C0F012036315811581742D75D1
:200D2B00F000C0E0C0F012036315811581743175F000C0E0C0F012036315811581743075AD
:200D4B00F000C0E0C0F012036315811581743075F000C0E0C0F01203631581158174DF75DF
:200D6B00F000C0E0C0F012036315811581744375F000C0E0C0F0120363158115812278FBDF
:200D8B0012001F8603088604748075F0701200B5120120758921F58DF58B75885975985263
:010DAB002225
:00000001FF
